:060000009031272B0000E7
:0800080083018031200077081C
:10001000A0007808A1007908A2007A08A300850151
:1000200091308400801C162891181F282008F700A2
:100030002108F8002208F9002308FA000900883195
:1000400000280B003F3406345B344F3466346D3483
:100050007D3407347F346F3477347C3458345E34E5
:10006000793471342200A2012208013C031C6B2860
:10007000220821006E072200A400003021006F3DFD
:100080002200A5002030A700A030A60022082607E5
:10009000F8000030273DFA00780884007A088500CF
:1000A0000008A6000B08F7008B132408230091001A
:1000B000220026082300930095131515553096004D
:1000C000AA309600951495186328151177088B04AB
:1000D0002200A20A34282000080022000D128D12EE
:1000E0008C012100EF01EE01200051082200A10047
:1000F000200050082200A000200032202100EF0143
:100100000230EE00200053082200A1002000520817
:100110002200A000200032202100EF010430EE0078
:10012000200055082200A100200054082200A00051
:10013000200032202100EF010630EE002000570899
:100140002200A100200056082200A000200032203A
:100150002100EF010830EE00200059082200A10024
:10016000200058082200A000200032202100EF01CA
:100170000A30EE0020005B082200A10020005A088F
:100180002200A000200032202100EF010C30EE0000
:1001900020005D082200A10020005C082200A000D1
:1001A000200032200B08F7008B130E302300910043
:1001B00020005E0823009300951315155530960016
:1001C000AA30960095149518E328151177088B042A
:1001D000003020002E1901302100EE000B08F7003E
:1001E0008B130F302300910021006E082300930031
:1001F0009513151555309600AA309600951495184C
:10020000FF28151177088B040B08F7008B131030AB
:10021000910020005F0823009300951315155530B9
:100220009600AA3096009514951814291511770890
:100230008B040B08F7008B1311309100200060082D
:10024000230093009513151555309600AA3096009B
:10025000951495182929151177088B040B08F700B8
:100260008B13123091002000610823009300951336
:10027000151555309600AA309600951495183E290C
:10028000151177088B04200008002B08D43E0318B2
:10029000672D2C3E732D2C08FC3E03189129043E3B
:1002A0006B2D0230AB0091290330AB0091295C0823
:1002B000D0025D08D13BD11B6429D108031D6729F9
:1002C0005008633C031C6729D1016430D0005108F9
:1002D000E3005008E20004302100A100B230A00089
:1002E000200091295C08D0075D08D13DD11B8729EA
:1002F0005108003C03188729FF3A031D8329500841
:10030000C23C031887290130D100C230D000510807
:10031000E3005008E20004302100A100B230A00048
:100320002000672DD101D0012E1C9A29AE189A29E0
:100330000230AC00AE102E18AE142C08023A03198D
:10034000A529013A0319B029B629AB016308D100E8
:100350006208D000EF01EE01ED01EC01F001B629D9
:100360000330AB006308D1006208D000672DD31FB3
:10037000BC29D11FC829BE29D11BCC295308510241
:10038000031CCC29031DC829500852020318CC298C
:100390005308D1005208D000E1080319D729730887
:1003A0006102031CDB2974086102031CDB292E1C7B
:1003B000DD29AE18DD290230AC00AE102E18AE14C7
:1003C0002C08023A0319E829013A0319002A062ADF
:1003D000AB016308D1006208D000EF01EE01ED012E
:1003E000EC01F001D408031DFF29D508031DFF29E6
:1003F000FF30EF00EE00E830ED008630EC00062A1A
:100400000330AB006308D1006208D000672D2C08D0
:10041000023A0319122A023A0319142A013A03195B
:10042000172A192AAB01192A1030AB00192A0430F7
:10043000AB00672D2C08023A0319252A023A03194A
:10044000282A013A03192B2A2D2A0530AB002D2A20
:100450000330AB002D2A0630AB00672D2C08023A82
:100460000319392A023A03193D2A013A03194B2A82
:100470005B2A6D200430AB005B2AD31B4A2AD308C9
:10048000031D462A5208643C03184A2A0A30D20245
:100490000030D33B5B2AD31B572A5308013C031C73
:1004A0005B2A031D572A5208C13C031C5B2A0A30F1
:1004B000D2070030D33D672D2C08023A0319672A72
:1004C000023A03196A2A013A03196D2A6F2A073082
:1004D000AB006F2A0430AB006F2A0830AB00672DE9
:1004E0002C08023A03197B2A023A03197F2A013A9F
:1004F00003198D2A992A6D200630AB00992AD51B45
:100500008C2AD508031D882A5408003C03188C2A1D
:1005100054080319D503D403992AD51B962AD50864
:10052000031D992A54081E3C031C992AD40A031956
:10053000D50A672D2C08023A0319A52A023A031995
:10054000A82A013A0319AB2AAD2A0930AB00AD2A1B
:100550000630AB00AD2A0A30AB00672D2C08023AFA
:100560000319B92A023A0319BD2A013A0319C62A06
:10057000D62A6D200830AB00D62A0A30D6020030C9
:10058000D73BD71FC52AD701D601D62A0A30D607AE
:100590000030D73DD71BD62AD708031DD32A5608CB
:1005A000783C0318D62AD7018230D600672D2C0854
:1005B000023A0319E22A023A0319E52A013A031919
:1005C000E82AEA2A0B30AB00EA2A0830AB00EA2A14
:1005D0000C30AB00672D2C08023A0319F62A023AB8
:1005E0000319FA2A013A03190C2B182B6D200A3033
:1005F000AB00182BD91F072B5908FE3C03180B2BF7
:10060000FF3A031D072B5808D83C03180B2B58083A
:100610000319D903D803182BD91B152BD908031D8F
:10062000182B5808273C031C182BD80A0319D90A81
:10063000672D2C08023A0319242B023A0319272BA1
:10064000013A03192A2B2C2B0D30AB002C2B0A302E
:10065000AB002C2B0E30AB00672D2C08023A03198F
:10066000382B023A03193C2B013A03193C2B432B3C
:100670006D200C30AB00432BDE08031D422B0130F4
:10068000DE00432BDE01672D2C08023A03194F2BA5
:10069000023A0319522B013A0319552B572B0F30ED
:1006A000AB00572B0C30AB00572B1030AB00672D35
:1006B0002C08023A0319632B023A0319672B013AFB
:1006C0000319672B752B6D200E30AB00752B5C0862
:1006D000053C031D722BDD08031D722BDD0101306B
:1006E000DC00752BDD010530DC00672D2C08023A9B
:1006F0000319812B023A0319842B013A0319872B22
:10070000892B1130AB00892B0E30AB00892B0330C5
:10071000AB00672D2C08023A0319952B023A0319F6
:10072000982B013A03199B2B9D2B1030AB009D2B6E
:100730002A30AB009D2B1230AB00672D2C08023AFB
:100740000319A92B023A0319AC2B013A0319AF2B59
:10075000B12B1330AB00B12B1130AB00B12B1430E7
:10076000AB00672D2C08023A031DB82B1230AB00EA
:10077000672D2C08023A0319C42B023A0319C72B20
:10078000013A0319CA2BCC2B1530AB00CC2B1230FD
:10079000AB00CC2B1630AB00672D2C08023A0319A6
:1007A000D82B023A0319DC2B013A0319EE2BFD2B4F
:1007B0006D201430AB00FD2BDB1BED2B5B08063CE2
:1007C0000318ED2BFF3A031DE92B5A08993C031837
:1007D000ED2B5A080319DB03DA03FD2BDB1BFA2B85
:1007E0005B08083C031CFD2B031DFA2B5A08663CD2
:1007F000031CFD2BDA0A0319DB0A672D2C08023AC9
:100800000319092C023A03190C2C013A03190F2C75
:10081000112C1730AB00112C1430AB00112C1830F8
:10082000AB00672D2C08023A031D182C1630AB00C4
:10083000672D2C08023A0319242C023A0319272C9D
:10084000013A03192A2C2C2C1930AB002C2C163011
:10085000AB002C2C1A30AB00672D2C08023A031D7C
:10086000332C1830AB00672D2C08023A03193F2CAB
:10087000023A0319422C013A0319452C472C1B302C
:10088000AB00472C1830AB00472C1C30AB00672D59
:100890002C08023A031D4E2C1A30AB00672D2C0891
:1008A000023A03195A2C023A03195D2C013A031932
:1008B000602C622C1D30AB00622C1A30AB00622C15
:1008C0001E30AB00672D2C08023A031D692C1C302A
:1008D000AB00672D2C08023A0319752C023A031954
:1008E000782C013A03197B2C7D2C1F30AB007D2C1A
:1008F0001C30AB007D2C2030AB00672D2C08023A59
:10090000031D842C1E30AB00672D2C08023A0319FE
:10091000902C023A0319932C013A0319962C982C27
:100920002130AB00982C1E30AB00982C2230AB004D
:10093000672D2C08023A031D9F2C2030AB00672D39
:100940002C08023A0319AB2C023A0319AE2C013AD7
:100950000319B12CB32C2330AB00B32C2030AB00E7
:10096000B32C2430AB00672D2C08023A0319BF2C9E
:10097000023A0319C32C013A0319C72CCB2C6D2062
:100980002230AB00CB2CE108031DE103CB2C610826
:100990004A3C0318E10A672D2C08023A0319D72CA8
:1009A000023A0319DA2C013A0319DD2CDF2C253029
:1009B000AB00DF2C2230AB00DF2C2630AB00672DE4
:1009C0002C08023A0319EB2C023A0319EF2C013AD6
:1009D0000319F42CF82C6D202430AB00F82C60089F
:1009E000083C0318E00AF82C6008033C031CE003F1
:1009F000672D2C08023A0319042D023A0319072D1A
:100A0000013A03190A2D0C2D2730AB000C2D243090
:100A1000AB000C2D2830AB00672D2C08023A0319CF
:100A2000182D023A03191C2D013A03191C2D1E2DF5
:100A30006D202630AB001E2D0430AE06672D2C082D
:100A4000023A03192A2D023A03192D2D013A0319EE
:100A5000302D322D2930AB00322D2630AB00322D17
:100A60002A30AB00672D2C08023A03193E2D023ABA
:100A70000319422D013A0319422D4B2D6D202830C8
:100A8000AB004B2D5F08323C031D492D3C30DF008D
:100A90004B2D3230DF00672D2C08023A0319572DF9
:100AA000023A03195A2D013A03195D2D5F2D2B309F
:100AB000AB005F2D2830AB005F2D1130AB00672DF0
:100AC0002C08023A031D662D2A30AB00672D043036
:100AD000AC008831282A0A148A100A15820757297F
:100AE0007229512954290A148A100A1582074B29A0
:100AF000B7299229072A1A2A2E2A5C2A702A9A2AAA
:100B0000AE2AD72AEB2A192B2D2B442B582B762BC8
:100B10008A2B9E2BB22BB92BCD2BFE2B122C192CF2
:100B20002D2C342C482C4F2C632C6A2C7E2C852C9D
:100B3000992CA02CB42CCC2CE02CF92C0D2D1F2D95
:100B4000332D4C2D602D2100CA014A08013C031CA5
:100B5000C72D2030D1007B30D0004A085007F80064
:100B60000030513DFA00780884007A0885004A0870
:100B70004807D2000030493DD300520823009100BD
:100B800095131514130880002100CA0AA52D4B08DF
:100B9000F8004C08F900200008000430F80021009B
:100BA0001D08833978049D000F30F8001F08F039C4
:100BB00078049F0022008D163530F700F70BDE2DEC
:100BC00021009D149D18E22D1B08C8001C08C900B7
:100BD00022008D12210049080E3C0318FA2DFF3A1D
:100BE000031DF62D4808A03C0318FA2D0130200003
:100BF000AD002100200008002030850078308400FE
:100C000000080319102E0A30F800F701F70B062E22
:100C1000F80B052E5F30F700F70B0C2E800B032E20
:100C20009031462D21004A0DF700F70DFC30F705F5
:100C30001D08833977049D000F30F8001F08F03934
:100C400078049F000D30F700F70B242E2000E401FC
:100C5000C701C60164080F3C031C3B2E21009D14F4
:100C60009D18302E1C08FA001B082000C6077A08C1
:100C7000C73DE40A2A2E210048088400490885005F
:100C80002000460880004708813F080021005608E0
:100C9000F700031023009517151400000000130837
:100CA00080000131910A0319920AF70B4C2E2000A3
:100CB000080020302100E500E101E201E301E40148
:100CC0005B08FA005A08F9005908F8005808F700BC
:100CD0000310771C792E5C08E1075D0803185D0F8F
:100CE000E2075E0803185E0FE3075F0803185F0F53
:100CF000E407E40CE30CE20CE10CFA0CF90CF80C40
:100D0000F70CE50B682E2000080083188B2E20308E
:100D100085008E3084002100550859068039E30093
:100D2000D51F9D2ED209D309D409D509D20A03199A
:100D3000D30A0319D40A0319D50AD91FAA2ED60932
:100D4000D709D809D909D60A0319D70A0319D80A25
:100D50000319D90AF701F801F901FA01DE01DF01EF
:100D6000E001E10159085804570456040319E82E1C
:100D70002030E2000310D20DD30DD40DD50DDE0DC1
:100D8000DF0DE00DE10D59086102031DD12E580859
:100D90006002031DD12E57085F02031DD12E560895
:100DA0005E02031CE22E5608DE025708031C570F92
:100DB000DF025808031C580FE0025908031C590FA2
:100DC000E1020314F70DF80DF90DFA0DE20BBA2E3E
:100DD000E31FF52EF709F809F909FA09F70A0319CB
:100DE000F80A0319F90A0319FA0A5E0880005F0875
:100DF000813F6008823F6108833F20000800103077
:100E00002100DC00F701FA01D90CD80C031C0E2FCD
:100E10005A08F7070318FA0A5B08FA07FA0CF70CE6
:100E2000F90CF80CDC0B042F2000080021005708F7
:100E300059068039DB00D71F222FD609D709D60AD9
:100E40000319D70AD91F292FD809D909D80A031994
:100E5000D90AF801F901F701FA015908031D332FE6
:100E6000580803194D2F1030DA000310D60DD70D96
:100E7000F70DFA0D59087A02031D402F5808770222
:100E8000031C492F5808F702031CFA035908FA02F9
:100E90000314F80DF90DDA0B352FDB1F542FF80969
:100EA000F909F80A0319F90A20000800210053087B
:100EB00055068039D700D31F622FD209D309D20A31
:100EC0000319D30AD51F692FD409D509D40A0319E8
:100ED000D50A1030D600F701FA01D30CD20C031C4E
:100EE000772F5408F7070318FA0A5508FA07FA0C7F
:100EF000F70CF90CF80CD60B6D2FD71F842FF809BF
:100F0000F909F80A0319F90A20000800F801F901A3
:100F1000F701FA0121004D08031D912F4C08031918
:100F2000AB2F1030CE000310CA0DCB0DF70DFA0D0C
:100F30004D087A02031D9E2F4C087702031CA72F31
:100F40004C08F702031CFA034D08FA020314F80DCB
:0A0F5000F90DCE0B932F20000800CE
:10100000F20A5F08323C031D0B287208173C0318D4
:101010000A28F20110287208133C03181028F20164
:10102000AE1D16282E181628F50118283308F500CD
:1010300022008C012000340803193428013A0319D6
:101040006F28033A0319AC28013A0319E628073A36
:1010500003191129013A03193929033A031961299E
:10106000013A03198D29CA29FE3022008E00750825
:101070000139F7002100EE017718EE172000320841
:101080000139F700F70EF70DF70DC030F7057708B7
:101090002100EE04200031080139F700F70EF70DAA
:1010A000E030F70577082100EE0420003008013910
:1010B000F700F70EF030F70577082100EE04200066
:1010C0002F080139F700F70DF70DF70DF830F70588
:1010D00077082100EE046E0822008C00CD29FD3037
:1010E00022008E0075080239F700770E2100EE000D
:1010F000EE0DEE0DC030EE05200032080239F7008B
:10110000F70EF70DE030F70577082100EE04200018
:1011100031080239F700F70EF030F70577082100A3
:10112000EE04200030080239F700F70DF70DF70D37
:10113000F830F70577082100EE0420002F08023967
:10114000F700F70DF70DFC30F70577082100EE04E6
:101150006E0822008C00CD29FB3022008E0075081D
:101160000439F700770E2100EE00EE0DE030EE05B9
:10117000200032080439F700F70EF030F705770841
:101180002100EE04200031080439F700F70DF70DB7
:10119000F70DF830F70577082100EE04200030083D
:1011A0000439F700F70DF70DFC30F705770821003B
:1011B000EE0420002F080439F7000310F70D77081C
:1011C0002100EE046E0822008C00CD29F7302200A9
:1011D0008E00200032080839F700770D2100EE005C
:1011E000EE0DEE0DF830EE05200031080839F7005D
:1011F000F70DF70DFC30F70577082100EE0420000D
:1012000030080839F7000310F70D77082100EE04C5
:1012100020002F0808392100EE046E0822008C00FF
:10122000CD29EF3022008E00200032081039F7005F
:10123000770D2100EE00EE0DFC30EE0520003108A8
:101240001039F7000310F70D77082100EE04200095
:10125000300810392100EE0420002F081039F70063
:101260000310F70C77082100EE046E0822008C00B2
:10127000CD29DF3022008E00200032082039F7000F
:101280000310770D2100EE002000310820392100E5
:10129000EE04200030082039F7000310F70C77081F
:1012A0002100EE0420002F082039F700F70CF70C7E
:1012B0003F30F70577082100EE046E0822008C000D
:1012C000CD29BF3022008E00200032084039210095
:1012D000EE00200031084039F7000310F70C7708C2
:1012E0002100EE04200030084039F700F70CF70C1D
:1012F0003F30F70577082100EE0420002F08403921
:10130000F700F70CF70CF70C1F30F70577082100F2
:10131000EE046E0822008C00CD297F3022008E0062
:101320002000320880392100EE0020006A08FF3AD0
:1013300021006E04F7000310770CEE002000310846
:1013400080392100EF0020006B08FF3A21006F0474
:10135000F700F70CF70C3F30F7057708EE04200094
:1013600030088039F700F70CF70CF70C1F30F70541
:1013700077082100EE0420002F088039F700F70ECF
:101380000F30F70577082100EE046E0822008C006C
:10139000CD292000FF3022008E002000B40A34083E
:1013A000083C031DDA292B08023C0319DA29B40191
:1013B0000830AE063408103C031DDF29B4018D1B34
:1013C000EC290D1BE729351FE7290130AC000D1F63
:1013D000EC29351BEC29AC010D08B500901DFD2949
:1013E000E708031DF629E8080319012AE808031D88
:1013F000012A6708473C031C012AE70A0319E80A87
:10140000032AE801E701901D0A2AE90803190A2ABC
:10141000E903152A9019152AE808031D132A6708FD
:10142000013C0318152A2430E900670B202AE8083C
:10143000031D202AE908031D202A0230AC00262AB9
:101440006808033C0318262A0330AC008031452984
:101450008831610873020318312A61087402031C81
:10146000332A2E18412AAB080319382A2B0B412A9C
:101470000130EC070318ED0A0319EE0A0319EF0A0D
:10148000462AEF01EE01ED01EC01F0016C0F592A43
:101490006D08193C031D592A6E0B592AEF08031DCC
:1014A000592AEF01EE01ED01EC01700F582A592A7B
:1014B000F00A6C0B772AED08031D772AEE08031D4E
:1014C000772AEF08031D772A54087002031D772A34
:1014D000D508031D772A54081F3C031D722AD5081E
:1014E0000319772AAB08031D772A0130AB006C0B78
:1014F000972AED08031D972AEE08031D972AEF0887
:10150000031D972A56087002031D972AD708031D4A
:10151000972A5608823C031D902AD7080319972A58
:10152000AB080319952A2B0B972A0230AB00210038
:10153000A008031D9E2AA1080319A22A2008031946
:10154000A103A003200BA92AA108031DA92A013089
:10155000F10020006A087F3C031DB32A2100A40A81
:101560000319A50A20006B087F3C031DBC2A21003B
:10157000A60A0319A70A20002100A80A0319A90A2C
:101580002808203C031DE22A2908033C031DE22A07
:10159000A901A801250CFA00240CF900FA0CF90C99
:1015A000FA0CF90C7908F300270CFA00260CF90064
:1015B000FA0CF90CFA0CF90C7908F400A501A40155
:1015C000A701A6012000911080311628E601E5014F
:1015D000E608031D2E2B6508143C031C2E2B21004E
:1015E0004908FA00480884007A0885000008CC0001
:1015F00001310008CD003F3103102000650DF900D6
:10160000660DFA007908703E2100CE003F307A3D29
:10161000CF004F082300920021004E0823009100C4
:10162000203085008030840002302100D6008031D7
:1016300020004626883121004D085102031C292B29
:10164000031D262B50084C020318292B20002E2B9B
:1016500021002000E50A0319E60AE82A0310650DB7
:10166000F900660DFA007908703E2100CC003F3089
:101670007A3DCD002300920021004C082300910008
:10168000203085001E30840002302100D6008031D9
:10169000200046268831013065022100CC00003050
:1016A0002000663B2100CD0003104C0DF9004D0DCC
:1016B000FA007908703ECC003F307A3DCD0023001F
:1016C000920021004C082300910020308500223038
:1016D000840002302100D600803120004626883167
:1016E0002100480884004908850001310008FA00FB
:1016F0003F31000820004202F7007A08433BF8001F
:101700000030443BF9000030453BFA002100CF0097
:101710007908CE007808CD007708CC000508D10004
:101720000408D000DB01DA01D9010A30D8004F08E3
:10173000DF004E08DE004D08DD004C08DC00803183
:101740002000592688312100510885005008840066
:101750007A082000B9007908B8007808B70077083F
:10176000B6003E084202F7003F08433BF80040083D
:10177000443BF9004108453BFA00BD007908BC0034
:101780007808BB007708BA00831039082100D5001B
:10179000200038082100D400200037082100D300A1
:1017A000200036082100D20020003D082100D90089
:1017B00020003C082100D80020003B082100D70071
:1017C00020003A082100D60080312000852688318B
:1017D0007A082100CF007908CE007808CD0077087C
:1017E000CC00063020006502F7000030663BFA00AE
:1017F00077082100D0007A08D100D9010A30D8003A
:101800005108DB005008DA0080312000FF268831C3
:101810007908FA00780821004C07F70079084D3D57
:10182000F80000304E3DF90000304F3DFA007808D6
:101830002000CF007708CE0021004A0884004B0822
:10184000850020004E0880004F08813F9031512EC6
:1018500021004908FA00480884004908850000086A
:10186000D20001310008D30001310008D400013159
:101870000008D5003D3120005A08F7005B08F80049
:10188000F901FA01DB1F462CF903FA0305082100D0
:10189000D7000408D6005508DB005408DA005308C6
:1018A000D9005208D8007A08DF007908DE007808ED
:1018B000DD007708DC0080312000592688312100C6
:1018C00057088500560884007A08D5007908D400A6
:1018D0007808D3007708D200CF01550CCE00540C05
:1018E000CD00530CCC00CE0CCD0CCC0CCE0CCD0CC2
:1018F000CC0C1F30CE052000E601E501E608031DF3
:10190000BC2C6508313C031CBC2C0310650DF90090
:10191000660DFA0079089A3E2100D2003F307A3DE8
:10192000D3005308230092002100520823009100A5
:10193000203085008430840002302100D6008031C0
:101940002000462688312100CF08031DB72CCE0881
:10195000031DB72C4D085502031CB72C031DB42CD6
:1019600054084C020318B72C2000BC2C2100200086
:10197000E50A0319E60A7E2C0310650DF900660DD1
:10198000FA0079089A3E2100D2003F307A3DD30018
:10199000230092002100520823009100203085008E
:1019A0001E30840002302100D600803120004626FF
:1019B0008831013065022100D20000302000663BF2
:1019C0002100D3000310520DF900530DFA007908DD
:1019D0009A3ED2003F307A3DD3002300920021008E
:1019E000520823009100203085002230840002300C
:1019F0002100D600803120004626883121004C0885
:101A000020004202F70021004D082000433BF8006F
:101A100021004E082000443BF90021004F0820001F
:101A2000453BFA002100D5007908D4007808D3009E
:101A30007708D200DB01DA01D9010A30D800550855
:101A4000DF005408DE005308DD005208DC0080315E
:101A50002000592688317A08B9007908B80078083A
:101A6000B7007708B6003E084202F7003F08433B44
:101A7000F8004008443BF9004108453BFA00BD002E
:101A80007908BC007808BB007708BA0083103908D1
:101A90002100D500200038082100D400200037089C
:101AA0002100D300200036082100D20020003D088C
:101AB0002100D90020003C082100D80020003B086C
:101AC0002100D70020003A082100D60080312000F4
:101AD000852688317A082100D5007908D400780855
:101AE000D3007708D200013020006502F7000030F3
:101AF000663BFA0077082100D6007A08D700D901A2
:101B00000A30D8005708DB005608DA008031200080
:101B1000FF2688317908FA0078082100D207790871
:101B2000D33D0030D43DD53D20004C08F7004D0892
:101B3000F800F901FA01CD1F9F2DF903FA032100E6
:101B40005208F7075308F83D5408F93D5508FA3D87
:101B500078082000CF007708CE005808CE02590838
:101B6000CF3B21004A0884004B08850020004E0826
:101B700080004F08813F080021004A08FC3E0318FE
:101B80001B2E043E2000252F3930B2000430B30054
:101B900002302100CD001B2E7130B2000430B300A2
:101BA00021004C08D3004B08D200D5010930D400E5
:101BB000803120005627883179082100D300780829
:101BC000D2005308D7005208D600D9010530D800FA
:101BD000803120001627883179082100CC00780850
:101BE000CB0020002B080B3C0319002E2B080F3CC8
:101BF0000319002E20302100CB070030CC3D2000FF
:101C00002100CC1B122E4C08023C0318122EFF3A66
:101C1000031D0E2E4B08E73C0318122E0330CC0098
:101C2000E730CB000230CD001B2EB3010330210082
:101C3000CD00200021004C08FA004B08CC1F282EB4
:101C40004B08003CF7000030FA004C08FA3B7708DC
:101C5000CE007A08CF000F304D0784002030850079
:101C60000318850A4F08D7004E08D600D9010A305C
:101C7000D800803120001627883177082100D40051
:101C80007A08D500FA0054088031200021208831DC
:101C9000F80080002100CD1B232F4D08003C0318C5
:101CA000232FCD0B882E4A08033C031D882E0F30AE
:101CB0004D078400203085000318850A4F08D7009F
:101CC0004E08D600D9010A30D800803120001627EE
:101CD000883179082100D5007808D4005508D7004C
:101CE0005408D600D9010A30D800803120001627C8
:101CF000883177082100D4007A08D500FA0054080A
:101D0000803120002120883180388000112F21006F
:101D10004F08D7004E08D600D9010A30D8008031CC
:101D200020001627883179082100D3007808D200D6
:101D3000D208031DA92ED308031DA92ECC1BA92E42
:101D40000F304D078400203085000318850A80017C
:101D5000122F4F08D7004E08D600D9010A30D800FC
:101D6000803120001627883179082100D3007808B7
:101D7000D200D208031DD12ED308031DD12ECE08C8
:101D8000031DC52ECF080319D12ECC1FD12E0F3025
:101D90004D078400203085000318850A40308000FC
:101DA000122FCE08031DE22ECF08031DE22ECC1FFA
:101DB000E22E0F304D078400203085000318850A7D
:101DC0008001122F0F304D0784002030850003184A
:101DD000850A4F08D7004E08D600D9010A30D8002E
:101DE000803120001627883179082100D500780835
:101DF000D4005508D7005408D600D9010A30D800BD
:101E0000803120001627883177082100D4007A0815
:101E1000D500FA0054088031200021208831F800D4
:101E2000800021004F08D7004E08D600D9010A30A3
:101E3000D800803120001627883179082100CF0092
:101E40007808CE004B2E200008000A148A140A15C8
:0A1E50008207C42DCC2D152E152E8F
:102000002B08D43E0318F22A2C3EF42A2D08023C59
:10201000031D1228AF01B0015430B1005830B20096
:10202000B3013528210020082104031929282000A4
:102030005E082100CA00200051082100CC002000C9
:1020400050082100CB0088312000BC259031352874
:10205000210020005E082100CA002308CC002208CD
:10206000CB0088312000BC259031F22A6D30AF00C2
:102070007830B0007C30B1006E30B200B301F22A8B
:102080002D08023C031D4C28AF01B0015430B100B3
:102090005830B200B30157285E082100CA00230857
:1020A000CC002208CB0088312000BC259031F22AD8
:1020B0007C30AF007730B0005830B100B200B301CF
:1020C000F22A6D30AF007930B0007830B1007C304A
:1020D000B200B301F22A5E082100CA0020005308B2
:1020E0002100CC00200052082100CB0088312000C4
:1020F000BC259031F22A5E30AF007930B000383024
:10210000B1007730B200B301F22A54081F3C031D1E
:102110009428D508031D9428AF015C30B0007130BD
:10212000B100B200B301A32802302100CA00200090
:1021300055082100CC00200054082100CB00883134
:102140002000BC259031F22A7330AF005C30B00023
:102150007130B100B200B301F22AD71BBE28D708F4
:10216000031DB6285608783C0318BE28AF015C3022
:10217000B0007130B100B200B301CD2802302100AF
:10218000CA00200057082100CC002000560821007A
:10219000CB0088312000BC259031F22A5C30AF00A2
:1021A0007130B0006D30B1007930B200B301F22A65
:1021B0005E082100CA00200059082100CC00200040
:1021C00058082100CB0088312000BC259031F22A2C
:1021D0003E30AF005430B0000430B1007830B2006F
:1021E000B301F22A5E082100CA00CC01CB0188317C
:1021F0002000BC259031F22A6D30AF007830B0005D
:102200007930B1007330B200B301F22A5E082100C8
:10221000CA0020005D082100CC0020005C082100DD
:10222000CB0088312000BC259031F22A5E30AF000F
:102230000430B0007730B1003D30B200B301F22A73
:102240007C30AF007730B0005830B100B200B3013D
:10225000F22A5830AF005C30B0003830B1005E3048
:10226000B200B301F22A5E082100CA0020004D0826
:102270002100CC0020004C082100CB008831200038
:10228000BC259031F22AAF015030B0007930B10056
:102290007130B200B301F22A03302100CA002000DD
:1022A0005B082100CC0020005A082100CB008831B7
:1022B0002000BC259031F22A7830AF006E30B0009B
:1022C0007330B1007930B200B301F22A2D0803193E
:1022D0007029013A03197A29033A031984298C29B0
:1022E0002A30AF001530B0005030B1007330B2006A
:1022F000B3018C292A30AF001530B0005030B10046
:102300007830B200B3018C29AF01B0015430B10074
:102310005830B200B3018C29F22A5030AF00793026
:10232000B000B1005E30B200B301F22A00302E18C6
:102330000130013A0319A029013A0319AA29B42945
:102340005C30AF007330B0007930B1005430B2006F
:10235000B301B4295830AF003830B0005C30B10060
:102360006D30B200B301B429F22A7830AF00583092
:10237000B000B1010630B200B301F22A5E082100BC
:10238000CA00200049082100CC0020004808210094
:10239000CB0088312000BC259031F22A7830AF0084
:1023A0005830B000B1015B30B200B301F22A5E08D0
:1023B0002100CA0020004B082100CC0020004A0860
:1023C0002100CB0088312000BC259031F22A5E30FC
:1023D000AF005830B000B1010630B200B301F22AAC
:1023E00002302100CA00CC017308CB0088312000E4
:1023F000BC259031F22A5E30AF005830B000B101F8
:102400005B30B200B301F22A02302100CA00CC01D5
:102410007408CB0088312000BC259031F22A0430AA
:10242000AF005E30B0003830B1007930B200B30197
:10243000F22AE108031D242AAF015C30B00071309C
:10244000B100B200B301302A02302100CA00CC0131
:10245000200061082100CB0088312000BC2590318C
:10246000F22A5E30AF005830B0003830B10004308E
:10247000B200B301F22A5F08323C031D752A210025
:10248000C901200060082100C8004908D900480897
:10249000D800DB016430DA0080312000FF26903163
:1024A0007908FA007808B03C2100C8000430C9005F
:1024B0007A08C93B4908CB004808CA00CD010C3056
:1024C000CC00803120008627903179082100C90096
:1024D0007808C8000230CA004908CC004808CB0080
:1024E00088312000BC259031AA2A60082100C8004C
:1024F0000A30C900F701F801480803104918F70726
:10250000F70CF80CC918F707F70CF80C4919F7077E
:10251000F70CF80CC919F707F70CF80C491AF7076C
:10252000F70CF80CC91AF707F70CF80C491BF7075A
:10253000F70CF80CC91BF707F70CF80C7808643C8B
:10254000C8000230CA00CC014808CB008831200006
:10255000BC259031F22A7330AF005C30B000B1007E
:102560005030B200B301F22A2E1DBE2AAF01B001D5
:102570005C30B1005430B200B301C52AAF015C3009
:10258000B0007130B100B200B301F22A7130AF0077
:102590005030B0007930B1006730B200B301F22A98
:1025A00002302100CA00CC0120005F082100CB00CE
:1025B00088312000BC259031F22A1C30AF007930E0
:1025C000B0005030B1006D30B200B301F22A0330D8
:1025D0002100CA00CC008E30CB0088312000BC2501
:1025E0009031F22A9031B12F0A108A140A11FB3E61
:1025F00003188A0A820006284028362858286128AD
:102600006B287B288528A428AD28CE28D828E82840
:10261000F228FC28062916292029292933294329AB
:102620004C295C2966298D299629B529BE29CE29F0
:10263000D729E729F029FB29042A0F2A192A312A48
:102640003B2AAB2AB42AC62AD02ADD2AE72AF03050
:10265000210099002000AB010430AC00AD012E1424
:10266000AE14B401B501B901B801B701B601BD019D
:10267000BC01BB01BA01C101C001BF01BE01C5015E
:10268000C401C301C201C701C601C901C801CB0110
:10269000CA01CD011930CC00CF01CE01E301E20126
:1026A000E401E601E501E801E701E901FF30EA00A4
:1026B000EB00EF01EE01ED01EC01F0010330210030
:1026C000A100E830A000A301A201F101F201A501DF
:1026D000A401A701A601F301F401A901A8012000AA
:1026E000AE11F50123008C018D018E0122009201B3
:1026F00091012000A501A6012100AB01AA01AF01B3
:10270000AE01AD01AC01B301B201B101B001B7013D
:10271000B601B501B401BB01BA01B901B801BD01EF
:10272000BC01BF01BE01C101C001C301C201C4019E
:10273000C5014610C610C7010830F8000638200051
:102740009C00D0309B0021009114C0308B040730D6
:102750008C00CF308D0000308E00901124008C0151
:10276000C0308D0021009513083024009000210016
:10277000951322000D128D122000B30121001E14AA
:102780009E141E11073023008C0009308D008A3002
:10279000220097002A0093012200980121001E12B6
:1027A0009E161E139E171D14C901C80180312000FA
:1027B000A32590317908D1007808D0002100C90103
:1027C0000230C80080312000A32590317908D30061
:1027D0007808D2002100C9010430C80080312000EF
:1027E000A32590317908D5007808D4002100C901CB
:1027F0000630C80080312000A32590317908D70029
:102800007808D6002100C9010830C80080312000B6
:10281000A32590317908D9007808D8002100C90192
:102820000A30C80080312000A32590317908DB00F0
:102830007808DA002100C9010C30C800803120007E
:10284000A32590317908DD007808DC000E302300E4
:1028500091009513151413082000DE000F3023009B
:102860009100951315141308F80020002E11781804
:102870002E15103023009100951315141308200015
:10288000DF00113023009100951315141308200068
:10289000E000123023009100951315141308200056
:1028A000E100D11B672CD108031D5A2C5008633C52
:1028B0000318672CD11B6B2C5108003C03186B2CA0
:1028C000FF3A031D672C5008C23C03186B2C0130E3
:1028D0002100C7002000D31B812CD308031D742CBA
:1028E0005208633C0318812CD31B852C5308003CF1
:1028F0000318852CFF3A031D812C5208C23C031893
:10290000852C01302100C7002000D51B902CD51B41
:10291000942CD508031D902C54081F3C0318942CAC
:1029200001302100C7002000D71B9F2CD71BA32CF0
:10293000D708031D9F2C5608823C0318A32C013096
:102940002100C7002000D91FAF2C5908FF3C031CF1
:10295000AF2C031DB82C5808D73C0318B82CD91B32
:10296000BC2CD908031DB82C5808283C0318BC2CD3
:1029700001302100C7002000DB1BD52C5B08073C81
:10298000031CC82C031DD52C5A08983C0318D52CC1
:10299000DB1BD92C5B08073C0318D92CFF3A031D1D
:1029A000D52C5A08673C0318D92C01302100C700E8
:1029B00020005C0BDE2CDD080319E92C5C08053CCB
:1029C000031DE52CDD080319E92C01302100C700A7
:1029D0002000DE080319F32C5E0BEF2CF32C0130E2
:1029E0002100C70020005F08323C0319FF2C5F085C
:1029F0003C3C0319FF2C01302100C7002000600877
:102A0000023C0318072D6008093C03180B2D013008
:102A10002100C700200061084B3C0318132D013032
:102A20002100C70020002100C7080319352D0130FF
:102A30002000D1007C30D000D301FA30D200D50183
:102A40000530D400D7011E30D600D901D801083096
:102A5000DB00DA01DD010530DC00DE012E11323051
:102A6000DF000530E000E101210020005108E30013
:102A70005008E2008031CD2590318031CD25903154
:102A80000A302100C80080312000FC2D9031AD01BA
:102A90008031CD25903122000D128D12FF302000A3
:102AA000EA00EB001A30F700F70B542D000021006C
:102AB0001E109E101E11073023008C0001308D0067
:102AC000C73021008D0022008D153030F800210024
:102AD0001D08833978049D000F30F8001F08F03975
:102AE00078049F000D30F700F70B742D9D149D188E
:102AF000772D1B08C2001C08C30022008D11CF30A7
:102B000021008D001E149E141E11073023008C001E
:102B100009308D00C3302A0093000830F8002100EE
:102B20001D08833978049D000F30F8001F08F03924
:102B300078049F000D30F700F70B9C2D9D149D1815
:102B40009F2D1B08BC071C08BD3D20002B08153C11
:102B50000319AD2D2A00930120005F08323C031DAC
:102B6000BB2D600872020319BA2D0C306007720287
:102B7000031DB12DC42D600872020319C42D0A3043
:102B800060077202031DBB2D60087202031DDE2D5B
:102B900020302100C9006030C8000130CA008031F7
:102BA00020001226903120302100C9005C30C8007E
:102BB000CA018031200012269031F62D20302100EC
:102BC000C9006830C8000130CA00803120001226D8
:102BD000903120302100C9006430C800CA01803122
:102BE0002000122690312100461420002100C61C2E
:102BF000002E2000AD018031CD2590312100C6107E
:102C000020002D08023C031D092E0230C9002B3084
:102C1000C800C91F0E2ED11F1A2E102ED11B202E18
:102C200049085102031C202E031D1A2E5008480289
:102C30000318202E7F30EA0022000D16232E2000DC
:102C4000FF30EA0022002000CB1F292ED11F352E95
:102C50002B2ED11B3D2E4B085102031C3D2E031D74
:102C6000352E50084A0203183D2E2D0B3D2E7F3085
:102C7000EB0022008D16402E2000FF30EB002200DA
:102C80002100C40A4408103C031D7E2E2030C900D8
:102C90006C30C8002030CB007030CA008831200072
:102CA000E62A90312100BD01BC01C11B612EC10883
:102CB000031D5E2E4008823C0318612EC1011E30A8
:102CC000C0004008BE074108BF3DC50A4508103C8A
:102CD000031D7D2EC5013F08D7003E08D600D9014F
:102CE0001030D80080312000162790317908CD00AF
:102CF0007808CC002100BF01BE01C401461CC52ECE
:102D000038083007C8003908313DC9003A08323D5B
:102D1000CA003B08333DCB0003104B0CB3004A0CF8
:102D2000B200490CB100480CB00034082C07C800B0
:102D300035082D3DC90036082E3DCA0037082F3D05
:102D4000CB0003104B0CAF004A0CAE00490CAD0099
:102D5000480CAC002030C9006030C8002030CB00E7
:102D60002A30CA00883120002824903120302100E8
:102D7000C9005C30C8002030CB002830CA00883140
:102D800020002824903121004610F1080319E52E77
:102D90002000AB080319CE2E2100E52EA4018B1BC9
:102DA000A4178B132100EF01EE012000510822002F
:102DB000A100200050082200A00080312000322015
:102DC0009031A41B8B17F10121002308D3002208A6
:102DD000D200D5011E30D40080312000562790311A
:102DE00078082100AA007908AB00200049082100DA
:102DF000D300200048082100D200D5010A30D400B9
:102E000080312000562790317908FA007808210097
:102E10002A07F8002B08FA3D7808AA007A08AB00C8
:102E20002B08CB002A08CA00CD012830CC00803105
:102E300020008627903178082100A2007908A3009D
:102E40002000500821002202C80020005108210063
:102E5000233BC900C91B332FC908031D4E2F480847
:102E6000023C031C4E2F2208200050022100C80003
:102E700023082000513B2100C900C91B462FC90867
:102E8000031D4E2F4808023C031C4E2F2000510802
:102E90002100A300200050082100A2004308013CAB
:102EA000031C6A2F031D582F4208373C031C6A2F4E
:102EB00020002E1D5E2FAD012E14682F2D08023C20
:102EC000031D672F2100C61420002E10682F2E101E
:102ED000AE2F21004308063C0318842FFF3A031D40
:102EE000752F4208063C0318842F4308083C031C36
:102EF000842F031D7F2F4208F93C031C842F2000E0
:102F0000AD012E14AE2F21004308083C03189F2F5B
:102F1000FF3A031D8F2F4208B13C03189F2F43082F
:102F20000B3C031C9F2F031D992F4208A43C031C3C
:102F30009F2F01302000AD002E14AE2F210043083A
:102F40000D3C0318AF2FFF3A031DAA2F4208A63CE1
:102F50000318AF2F02302000AD002E1421002000F6
:102F600000285F08323C031DBD2FF2080319BC2F57
:102F700072080C3C031DB52FC42FF2080319C42F8F
:0C2F800072080A3C031DBD2F4B2D63009E
:107EE00006345734A1345C345D346234FB34673477
:107EF00077346D34F43472344334783474347D34EC
:107F0000833482345C3487341C348C34A63490340B
:107F1000FA3494343034993432349D340B34A134EF
:107F2000BC34A4342E34A8345134AB340E34AE34C3
:107F30004634B03400340034EB340334EC340734CA
:107F400001340C342A34103467341434B734183400
:107F500019341D348C3421340F342634A3342A349C
:107F600045342F34F6343334B534383481343D3429
:107F70005A3442343E3447342D344C342634513450
:107F80002934563435345B344934603464346534D0
:107F900087346A34AF346F34DC3474340F347A3459
:107FA00045347F347E348434BA348934F8348E34A2
:107FB0003734943476349934B5349E34F334A3345E
:107FC0002F34A9346934AE34A034B334D334B83444
:107FD0000234BE342B34C3344F34C8346C34CD3403
:107FE0008134D2348F34D7349434DC348F34E13458
:107FF0008034E6346734EB344234F0341034F534F2
:020000040001F9
:04000E00840FFF1A42
:00000001FF
